:1000000012C02AC029C028C027C026C025C024C0CD
:1000100023C022C021C020C01FC01EC01DC01CC0E4
:100020001BC01AC019C011241FBECFEDCDBF10E0F8
:10003000A0E6B0E0E6EEF1E002C005900D92A03639
:10004000B107D9F710E0A0E6B0E001C01D92A437D7
:10005000B107E1F74AD0C6C0D3CFAC01892B59F024
:1000600020E030E08AEF90E00197F1F72F5F3F4FFB
:1000700024173507B9F70895D19A8A9A8D988B9AE3
:100080008C9AB89A089582E08BB98CE089B980E1A6
:100090008AB90895939AD99A929880B3949A0895B8
:1000A0009298939820E092989298992314F4D99A70
:1000B00001C0D998929A929A2F5F203119F0880F37
:1000C000991FF1CF9298939A089590E08599FECF69
:1000D000859BFECF882314F4949A01C094989F5F67
:1000E000983010F4880FF2CF0895CF92DF92EF92FC
:1000F000FF921F93CF93DF93BFDFCCDFC4DFC09AA3
:1001000084E690E0AADF80E09CECCADF82E790E919
:10011000C7DF80E496EAC4DF80E490EDC1DF81E1CF
:1001200098ECBEDF80E292ECBBDF81E090ECB8DFC0
:1001300080E090EBB5DF0F2EF0E6EF2EF0E0FF2E23
:10014000F02D0F2EF4E1CF2EDD24F02DCE0CDF1C90
:10015000C09880E18AB95F9BFECF8CB1809360002C
:100160008FEF91E001C08FEF5F9903C08150E1F7FD
:1001700002C0882319F4943138F00EC08CB1F70115
:10018000E90FF11D808308C0F701E90FF11D10820E
:100190009F5F943121F0F8CF9F5F943120F38CB1B1
:1001A0005498C09A89E390EC7BDF10E08AEA8DDFF7
:1001B0001F5F1330D9F78DE288DF84ED86DFE7011A
:1001C00010E0888182DF8991180FCC15DD05C9F711
:1001D000812F7BDF8AEA79DF8AEA77DF81E090ECA2
:0601E0005FDFB6CFFFCF88
:00000001FF
